:10000000A401DC2890002808840026086E208413B0
:100010000005181C2606031920281008031D18289F
:100020001608FF3E031C21280A30832016082128C9
:10003000100AFF3003192028100B20281708212848
:100040009909990CD728A416A41EA41224192D28A6
:10005000FE39A50024150310D728241A352892004C
:1000600024164C2003183A281208532003183A2863
:10007000A41ED72845206A2024112412A411280880
:1000800084002608841780044B2828088400260949
:1000900080058417800508003F206A2045206620DF
:1000A0002508A41901388E0008308F008E0D031822
:1000B0003F20031C45206A2066208F0B56283F20D6
:1000C0006A202808840026080005FF3E29088400CD
:1000D0002709482829088400270842288417800413
:1000E000D72889008316081483120808D7288800A7
:1000F0008316081555308900AA308900881488189D
:100100007F280811D7288F018E00FF308E07031C2F
:100110008F07031CD72803308D00DF3091208528FE
:100120008D01E83E8C008D09FC30031C9A288C0759
:10013000031897288C0764008D0F97280C18A028A7
:100140008C1CA4280000A42808008D018F018E00BB
:100150000230AD288E000630AD2894000F080D0245
:10016000031DB4280E080C020430031801300319D3
:1001700002301405031DFF30D7280404031DFF308F
:10018000D728103094008D018C01930C920C031C25
:10019000CF280E088C070F0803180F0F8D078D0C42
:1001A0008C0C910C900C940BC5281008D728831345
:1001B000031383126400080083168617861506163B
:1001C00086160617051185118312C230B000003063
:1001D0007120B80001307120B90002307120BA00DE
:1001E00003307120BB00380892009301E8308E0084
:1001F00003308F00C1209E0011089F003908920033
:10020000930164308E008F01C120A0001108A1006D
:100210001E08A0071F080318013EA1073A08920014
:1002200093010A308E008F01C120A2001108A300A3
:100230002008A20721080318013EA3073B08220754
:10024000AC0023080318013EAD002C08AA002D08BD
:10025000AB000830920093012C088E002D088F000F
:10026000C120AE001108AF00B101B201B3010330EB
:100270008F00E83084203923BD010630A80080308B
:10028000A60001309800FF309600970101309900D8
:1002900031080220B1000318582914308320BD0A08
:1002A000640032303D02031C5729BD0139233D292A
:1002B00086193C14861D3C10061ABC14061EBC1080
:1002C000861A3C15861E3C11061BBC15061FBC1168
:1002D0000230BC1C03019E000030BC1C03019F00C7
:1002E00003013C1801309E0703189F0A04303C1D8F
:1002F0000301A00000303C1D0301A1001E08A0075F
:100300001F080318013EA1070830BC1D0301A2000D
:100310000030BC1D0301A30020082207B4006400C4
:100320003408023C031D962998299829BD013D29CE
:10033000B30164004B3033020318B2290630A80021
:100340008030A60001309800FF3096009701013000
:10035000990031080220B1000318B4291430832019
:10036000B30A9929BD013D2986193C14861D3C100C
:10037000061ABC14061EBC10861A3C15861E3C11BB
:10038000061BBC15061FBC110230BC1C03019E00DD
:100390000030BC1C03019F0003013C1801309E0784
:1003A00003189F0A04303C1D0301A00000303C1DCF
:1003B0000301A1001E08A0071F080318013EA107A2
:1003C0000830BC1D0301A2000030BC1D0301A300C6
:1003D00020082207B50035088C000330A5209E00B8
:1003E00035088C000430A520A0001E0884002008D9
:1003F000BD20A000A1006400200821040319022AE6
:10040000042A042ABD013D29B30164004B303302A4
:1004100003181E2A0630A8008030A600013098007C
:10042000FF30960097010130990031080220B10099
:100430000318202A14308320B30A052ABD013D2960
:1004400086193C14861D3C10061ABC14061EBC10EE
:10045000861A3C15861E3C11061BBC15061FBC11D6
:100460000230BC1C03019E000030BC1C03019F0035
:1004700003013C1801309E0703189F0A04303C1DFD
:100480000301A00000303C1D0301A1001E08A007CD
:100490001F080318013EA1070830BC1D0301A2007C
:1004A0000030BC1D0301A30020082207B600640031
:1004B0003608003C031D5E2ABD013D2964000C3056
:1004C0003602031C652ABD013D29640036080A3C3A
:1004D000031D6B2AB6016C2AB30164004B30330252
:1004E0000318862A0630A8008030A6000130980044
:1004F000FF30960097010130990031080220B100C9
:100500000318882A14308320B30A6D2ABD013D29BF
:1005100086193C14861D3C10061ABC14061EBC101D
:10052000861A3C15861E3C11061BBC15061FBC1105
:100530000230BC1C03019E000030BC1C03019F0064
:1005400003013C1801309E0703189F0A04303C1D2C
:100550000301A00000303C1D0301A1001E08A007FC
:100560001F080318013EA1070830BC1D0301A200AB
:100570000030BC1D0301A30020082207B70064005F
:100580003708003C031DC62ABD013D2964000C301C
:100590003702031CCD2ABD013D29640037080A3CFF
:1005A000031DD32AB701D42A3408B8003508B9008E
:1005B0003608BA003708BB00380892009301E830CB
:1005C0008E0003308F00C1209E0011089F00390863
:1005D0009200930164308E008F01C120A0001108A9
:1005E000A1001E08A0071F080318013EA1073A0832
:1005F000920093010A308E008F01C120A2001108E1
:10060000A3002008A20721080318013EA3073B0806
:100610002207AC0023080318013EAD002C088C0013
:100620002D088D0009308F009230AA20031D1A2B4F
:10063000BD013D290830920093012C088E002D0841
:100640008F00C120AE001108AF002C088C002D08CF
:100650008D002B088F002A08A720031D342B4C2364
:100660002C08AA002D08AB003923BD013D296300E9
:10067000372B0530A8000830A6000530A90004304B
:10068000A700300825202F0825202E0825208E3091
:100690002320143083200800890138087720013096
:1006A000890039087720023089003A087720033022
:0806B00089003B0877200800D7
:02400E00F53F7C
:084200000200030000000800A9
:00000001FF
